:100000000C94AB020C94C6020C94C6020C94C6026B
:100010000C94C6020C94C6020C94C6020C94C60240
:100020000C94C6020C94C6020C94C6020C94C60230
:100030000C94C6020C94F50A0C941E0B0C94C60288
:100040000C94C6020C94C6020C94C6020C94C60210
:100050000C94C6020D5363616E6E696E6720427523
:100060007320666F7220445331385832300D004E81
:100070006F2053656E736F7220666F756E640D002E
:10008000427573204572726F720D002E003000B001
:1000900043205B002E00B0435D000D4453313858BF
:1000A000323020312D576972652D52656164657259
:1000B0002044656D6F206279204D617274696E20F5
:1000C00054686F6D61730D002D2D2D2D2D2D2D2D4F
:1000D0002D2D2D2D2D2D2D2D2D2D2D2D2D2D2D2D50
:1000E0002D2D2D2D2D2D2D2D2D2D2D2D2D2D2D2D40
:1000F0002D2D2D0020445331385832302053656E59
:10010000736F7228732920617661696C61626C6516
:100110003A0D002320696E20427573203A00203A80
:1001200020000D0053656E736F72232000206973E9
:1001300020612000445331385332302F445331383A
:1001400032300044533138423230002077686963DE
:10015000682069732000706172617369746500655D
:10016000787465726E616C6C790020706F7765725F
:1001700065640D000D4453313878323020454550C8
:10018000524F4D20737570706F7274207465737464
:1001900020666F7220666973742073656E736F7268
:1001A0000D0054482F544C2066726F6D2045455009
:1001B000524F4D2073656E736F722031203A2000CC
:1001C000202F20000D0054482B3120616E642054F4
:1001D0004C2B31207772697474656E20746F2073B4
:1001E0006372617463687061640D0073637261743B
:1001F000636870616420636F7069656420746F2048
:100200004453313878323020454550524F4D0D001F
:100210004453313878323020454550524F4D206399
:100220006F70696564206261636B20746F20736313
:1002300072617463687061640D00544820616E647B
:1002400020544C2076657269666965640D00766598
:1002500072696679206661696C65640D0054482F87
:10026000544C2066726F6D20454550524F4D20739F
:10027000656E736F722031206E6F77203A200020F8
:100280002F20000D000D5468657265206973206F82
:100290006E6C79206F6E652073656E736F72202DA2
:1002A0003E2044656D6F206F662022726561645F39
:1002B0006D6561735F73696E676C65223A0D000D41
:1002C000000D436F6E766572745F5420616E64201A
:1002D000526561642053656E736F7220627920539A
:1002E000656E736F72202872657665727365206F14
:1002F00072646572290D0053656E736F722320005E
:10030000203D2000435243204572726F7220286CBA
:100310006F737420636F6E6E656374696F6E3F29CF
:10032000000D005374617274206D6561732E206638
:1003300061696C6564202873686F727420636972E8
:10034000637569743F29000D436F6E766572745F43
:100350005420666F7220616C6C2053656E736F72EF
:100360007320616E6420526561642053656E736F03
:10037000722062792053656E736F720D0053656E43
:10038000736F72232000203D2000435243204572AA
:10039000726F7220286C6F737420636F6E6E65636A
:1003A00074696F6E3F29000D005374617274206D83
:1003B0006561732E206661696C6564202873686FBF
:1003C000727420636972637569743F29000D566504
:1003D00072626F7365206F75747075740D002E00F6
:1003E0003000B0430046433A004352433A00534E74
:1003F0003A2000200028313853290028313842297A
:100400000028203F20290020435243204641494CE8
:10041000200020435243204F2E4B2E200053503AB1
:10042000004352433A0020004E6F2053656E736FB5
:100430007220666F756E640D00427573204572728E
:100440006F720D0020435243204641494C2000204A
:10045000435243204F2E4B2E200020545F72617771
:100460003D0020005332302F3039004232302F31DE
:1004700032004232302F313100204232302F3130C1
:1004800020004232302F30390020000D004453311B
:10049000385832305F73746172745F6D6561733A9E
:1004A0002053686F727420436972637569742021E8
:1004B0000D00445331385832305F77726974655F8C
:1004C000736372617463687061643A2053686F7219
:1004D00074204369726375697420210D004453319F
:1004E000385832305F726561645F73637261746340
:1004F000687061643A2053686F7274204369726354
:1005000075697420210D00445331385832305F63CF
:100510006F70795F736372617463687061643A20AD
:1005200053686F7274204369726375697420210D7A
:1005300000445331385832305F726563616C6C5FD0
:1005400045323A2053686F7274204369726375694B
:100550007420210D000011241FBECFE5D8E0DEBFBE
:10056000CDBF10E0A0E6B0E0E4EAF8E102C00590FB
:100570000D92AA36B107D9F710E0AAE6B0E001C0A3
:100580001D92AE3DB107E1F70C948F030C9400006F
:100590001F93CF93DF93CDB7DEB729970FB6F894AB
:1005A000DEBF0FBECDBF84E590E00E94940B10E04B
:1005B0008FEF8987BE016F5F7F4FCE0109960E9442
:1005C0003F0929852F3F19F48FE690E004C02E3FA4
:1005D00029F480E890E00E94940B16C0E12FFF27D9
:1005E00083E0EE0FFF1F8A95E1F7E155FF4FDE0133
:1005F000119697E08D918193915097FFFBCF1F5FEC
:10060000222311F01530B0F2812F992729960FB6C9
:10061000F894DEBF0FBECDBFDF91CF911F9108953B
:10062000EF92FF920F931F93CF93DF93CDB7DEB777
:1006300061970FB6F894DEBF0FBECDBF182FE62E20
:10064000F42E882311F08DE201C08BE20E94730B1F
:100650008E2D99270E94A60B8BE890E00E94940BA8
:100660002F2D33274AE050E0BE016F5F7F4F81E7B7
:1006700092E0289FF001299FF00D389FF00D112482
:10068000CF010E94F60BDE011196FD0101900020C2
:10069000E9F73197EA1BFB0B84E08E1B39F0082F3A
:1006A0008DE890E00E94940B0150D1F7CE010196A5
:1006B0000E94850B8FE890E00E94940B112311F0AB
:1006C0008DE201C08BE20E94730B4F2D6E2D812FA6
:1006D0000E94D8088C016AE070E00E942B0CCB01CC
:1006E0000E94A60B84E990E00E94940BC8016AE086
:1006F00070E00E942B0C805D0E94730B86E990E0F5
:100700000E94940B61960FB6F894DEBF0FBECDBF6A
:10071000DF91CF911F910F91FF90EF900895C3E566
:10072000D8E0DEBFCDBF89E190E00E94440B26E017
:1007300041E350E062E370E080E390E00E94A505B1
:1007400078948AE990E00E94940B88EC90E00E94F3
:10075000940B0E94C802E82E99270E94A60B84EFF2
:1007600090E00E94940BEE2021F13FEAC32E30E08E
:10077000D32E00E010E0FE2C83E191E00E94940B68
:100780000F5F1F4FC8010E94A60B8EE191E00E94EF
:10079000940B68E070E0C6010E94290782E291E0B4
:1007A0000E94940BFA9428E030E0C20ED31EFF2082
:1007B00019F7EE20E9F10FEA10E05801CC24DD240E
:1007C000FE2C84E291E00E94940BC60101960E94E7
:1007D000A60B8DE291E00E94940BF501808128E048
:1007E00030E0A20EB31E803119F484E391E002C020
:1007F00083E491E00E94940B8BE491E00E94940BBF
:10080000C8010E945C09882319F486E591E002C0C2
:100810008FE591E00E94940B8AE691E00E94940B90
:10082000FA940894C11CD11C085F1F4FFF2049F6A1
:10083000EE2009F469C084E791E00E94940BBE01A8
:100840006F5F7F4F8FEA90E00E94860A1B810C81C8
:1008500082EA91E00E94940B812F99270E94A60BB7
:1008600080EC91E00E94940B802F99270E94A60BA8
:1008700084EC91E00E94940B0F5F1F5F20E6402FF5
:10088000612F8FEA90E00E94580A86EC91E00E9466
:10089000940B6FEA70E080E00E94AC0A8BEE91E06E
:1008A0000E94940B8FEA90E00E94D60A80E192E0C9
:1008B0000E94940BBE016F5F7F4F8FEA90E00E9411
:1008C000860A8B81181731F48C81081719F48AE392
:1008D00092E002C08EE492E00E94940B1B810C8196
:1008E0008DE592E00E94940B812F99270E94A60B20
:1008F0008FE792E00E94940B802F99270E94A60B0D
:1009000083E892E00E94940B31E0E31631F585E82C
:1009100092E00E94940BF090AF0060E070E080E005
:100920000E94740966E471E48FE090E00E94B306CF
:100930009E01265F3F4FAE01455F5F4FBE01645F82
:100940007F4F8F2D0E94F8094A856B858C850E9408
:1009500010038FEB92E00E94940B81EC92E00E94D6
:10096000940BFE2CFF2009F442C0CF2CDD2486011D
:1009700023E0000F111F2A95E1F709551F4FB80119
:1009800080E00E947409882361F566E471E48FE0D9
:1009900090E00E94B30687EF92E00E94940BC6019C
:1009A0000E94A60B80E093E00E94940B9E01265FBC
:1009B0003F4FAE01455F5F4FBE01645F7F4FC8018F
:1009C0000E949409882331F44A856B858C850E94A6
:1009D000100304C084E093E00E94940B81E293E052
:1009E00002C083E293E00E94940BFA94BBCF87E4A9
:1009F00093E00E94940B60E070E080E00E94740934
:100A0000182F882309F041C066E471E48FE090E07C
:100A10000E94B3061E15E8F59FEAC92E90E0D92E74
:100A200000E010E0FE2C8DE793E00E94940BC801DB
:100A300001960E94A60B86E893E00E94940B9E010B
:100A4000265F3F4FAE01455F5F4FBE01645F7F4F42
:100A5000C6010E949409882331F44A856B858C85F0
:100A60000E94100304C08AE893E00E94940B87EA76
:100A700093E00E94940BFA940F5F1F4F88E090E080
:100A8000C80ED91EFF2079F604C089EA93E00E94BF
:100A9000940B8DEC93E00E94940B60E070E080E09A
:100AA0000E94740966E471E48FE090E00E94B3064E
:100AB0000E94000868E175E08DE390E00E94B306B3
:100AC0004CCFE091D700F091D8009091D90090954B
:100AD000808189238083E091DC00F091DD008081BA
:100AE0009091D900892B80838FEB93E0811591053C
:100AF00011F00197F1F73FB7F894E091DC00F09125
:100B0000DD009091D900909580818923808383E8CE
:100B100090E08115910511F00197F1F7E091DA006D
:100B2000F091DB0040812091D90042233FBF8BE34D
:100B300093E08115910511F00197F1F780818223EF
:100B400009F441E0842F992708955093DD004093E4
:100B5000DC007093D8006093D7009093DB00809303
:100B6000DA0081E090E002C0880F991F2A95E2F731
:100B70008093D9000E9461050895E091DA00F09118
:100B8000DB0080819091D900892399270895E09115
:100B9000D700F091D80080819091D900892B808373
:100BA000E091DC00F091DD0080819091D900892BEB
:100BB00080830895E091D700F091D8009091D900FA
:100BC0009095808189238083E091DC00F091DD00A5
:100BD0009091D90090958081892380830895382F42
:100BE0004FB7F894E091DC00F091DD0080819091A6
:100BF000D900892B808381E090E08115910511F067
:100C00000197F1F7332351F0E091DC00F091DD0022
:100C10009091D900909580818923808389E190E02B
:100C20008115910511F00197F1F7E091DA00F0914B
:100C3000DB00E0812091D900E22309F43E2F89E511
:100C400090E08115910511F00197F1F7E091DC003A
:100C5000F091DD0020958081822380834FBF832F18
:100C6000992708951F93CF93C82F18E08C2F817078
:100C70000E94EF05C6958111C0681150B9F78C2FFD
:100C80009927CF911F9108958FEF0E9432069927DF
:100C90000895DF92EF92FF920F931F93CF93DF930C
:100CA000E82EEB010E946105182F882319F08FEFC1
:100CB00090E032C080EF0E943206D12E00E488E03E
:100CC000F82E81E00E94EF05182F81E00E94EF05C9
:100CD000882329F0112371F08EEF90E01DC01123BD
:100CE00049F40E1528F0888180FF04C0E01611F049
:100CF00011E0D02E812F0E94EF0588818695888390
:100D0000112311F0806888830150FA94D1F621965E
:100D10000023A9F68D2D9927DF91CF911F910F9177
:100D2000FF90EF90DF9008950F931F93CF93DF9381
:100D3000082FEB010E946105209751F085E50E9484
:100D4000320618E089910E9432061150D9F703C08B
:100D50008CEC0E943206802F0E943206DF91CF91E8
:100D60001F910F910895DC01CB0181159105A1051B
:100D7000B10529F081509040A040B040D9F70895C6
:100D8000EF92FF920F931F93CF93DF93CDB7DEB710
:100D900061970FB6F894DEBF0FBECDBF162F042F9C
:100DA000882311F08DE201C08BE20E94730B812F2A
:100DB00099270E94A60B8EED93E00E94940B202FA2
:100DC00033274AE050E0BE016F5F7F4F81E792E03A
:100DD000289FF001299FF00D389FF00D1124CF01BD
:100DE0000E94F60B8E010F5F1F4FF801019000204B
:100DF000E9F73597EE24FF24E017F107A9F080EE1C
:100E000093E00E94940B0894E11CF11CF8010190FE
:100E10000020E9F73197E01BF10B84E090E08E1B96
:100E20009F0BE816F90658F3CE0101960E94850B38
:100E300082EE93E00E94940B61960FB6F894DEBFA9
:100E40000FBECDBFDF91CF911F910F91FF90EF901B
:100E50000895CF92DF92EF92FF920F931F93CF935B
:100E6000DF936C017B01C0E0D0E0C617D707B0F577
:100E70008C01209719F485EE93E007C0C701019714
:100E8000C817D90721F489EE93E00E94940BC13072
:100E9000D10521F48EEE93E00E94940BF80180813D
:100EA0000E94CB0B83EF93E00E94940B209781F478
:100EB000F6018081803119F485EF93E007C0883214
:100EC00019F48BEF93E002C081E094E00E94940B50
:100ED00021960F5F1F4FCE15DF0558F268E070E0D6
:100EE000C6010E94D60B882319F087E094E002C067
:100EF00082E194E00E94940BDF91CF911F910F91BA
:100F0000FF90EF90DF90CF900895EF92FF920F93B4
:100F10001F93CF93DF937C01EB018DE194E00E945E
:100F2000940B00E010E00C171D07B8F4CE010197F8
:100F30000817190721F481E294E00E94940BF7014D
:100F400081917F010E94CB0B86E294E00E94940B7A
:100F50000F5F1F4F0C171D0748F3DF91CF911F91B3
:100F60000F91FF90EF9008950F931F93CF93C82F89
:100F7000FB01DA01A9018081282F3327818199277C
:100F8000982F8827282B392BC03159F42E7F63E006
:100F9000220F331F6A95E1F78681281B3109245FF0
:100FA0003F4F37FF06C081E08C93309521953F4F2E
:100FB00001C01C92C83291F48481682F7727CB013D
:100FC000807690708036910549F066FF02C02E7FD2
:100FD00005C065FF02C02C7F01C0287FC90134E035
:100FE000969587953A95E1F7FA018083822F8F7065
:100FF000F801808380E090E0CF911F910F910895D8
:10100000DF92EF92FF920F931F93CF93DF93CDB7B1
:10101000DEB765970FB6F894DEBF0FBECDBFBFEF4A
:10102000DB2EBE016F5F7F4F8D2D0E944906D82EAB
:101030008FEFD81639F488E294E00E94940B8FEF7A
:1010400090E0A8C0EEEFDE1639F489E394E00E9448
:10105000940B8EEF90E09EC068E070E0CE010196A8
:101060000E9429078981883219F0803109F089C0EE
:101070008DE00E94730B8EEB0E943206EE24FF245B
:1010800098E08E010F5F1F4F0E0D1F1D9D8B0E945C
:101090004406F80180879D8991500894E11CF11C59
:1010A00097FFEFCFA9E0EA2EF12CEC0EFD1E69E0D0
:1010B00070E0C7010E94850769E070E0C7010E94E7
:1010C000D60B882319F084E494E002C08FE494E006
:1010D0000E94940B8DE00E94730B8985082F1127C5
:1010E0008A859927982F8827082B192B8AE594E061
:1010F0000E94940B812F99270E94CB0B802F0E9476
:10110000CB0B82E694E00E94940B8981803119F424
:1011100084E694E01AC08832D1F49D85292F3327C4
:10112000C901807690708036910519F48BE694E0C1
:101130000CC026FF03C082E794E007C025FF03C070
:1011400089E794E002C082E894E00E94940B89E869
:1011500094E00E94940B8E010E5E1F4F9E012D5E47
:101160003F4FAE014C5E5F4FB70189810E94B407CB
:101170004A896B898C890E94C00680E690E00E94B3
:10118000850BDD2009F04DCF8BE894E00E94940B95
:1011900080E090E065960FB6F894DEBF0FBECDBF3D
:1011A000DF91CF911F910F91FF90EF90DF90089505
:1011B000EF92FF920F931F93CF93DF93CDB7DEB7DC
:1011C00028970FB6F894DEBF0FBECDBF082F162F9D
:1011D0007E010894E11CF11C88E0E2E6F0E0D70112
:1011E00001900D928A95E1F7242F332781E792E051
:1011F000289FB001299F700D389F700D1124CB01DD
:1012000068EE73E00E943F0C8AE0189FC001112431
:10121000680F791F002359F4902FF7018191481727
:1012200019F46F5F7F4F03C09F5F9830B8F3CB0115
:1012300028960FB6F894DEBF0FBECDBFDF91CF91D9
:101240001F910F91FF90EF900895882319F07095EA
:1012500061957F4F442319F0309521953F4F6217D8
:1012600073071CF48FEF9FEF0895261737071CF4C0
:1012700081E090E0089580E090E0089508950F9354
:101280001F93CF93DF938C01EB01BE01F8018081A6
:101290000E944906982FF80180838E5F823038F0D3
:1012A000992329F08881883211F0803171F7DF911C
:1012B000CF911F910F9108950F931F938C010E945E
:1012C0006105B80184EB0E94940681E00E94EF055D
:1012D000182F0E94610580E090E0112311F081E059
:1012E00090E01F910F9108951F93CF93DF93182FD4
:1012F000EB010E9461050E94BD05882359F0BE01E3
:1013000084E40E949406113011F00E94C70580E029
:1013100090E006C08DE894E00E94940B82E090E09B
:10132000DF91CF911F9108952F923F924F925F923C
:101330006F927F928F929F92BF92CF92DF92EF92A5
:10134000FF920F931F93CF93DF93CDB7DEB729970B
:101350000FB6F894DEBF0FBECDBF4C011B012A01B2
:1013600039010E946105B4018EEB0E949406EE24BF
:10137000FF2418E0B12E6E010894C11CD11C870116
:101380000C0D1D1D0E944406F8018083BA94089438
:10139000E11CF11CB7FEEFCF69E070E0C6010E94CE
:1013A000D60B882319F083E090E00AC083019201F4
:1013B000A101B601F40180810E94B40780E090E0B1
:1013C00029960FB6F894DEBF0FBECDBFDF91CF9147
:1013D0001F910F91FF90EF90DF90CF90BF909F9063
:1013E0008F907F906F905F904F903F902F900895D7
:1013F0004F925F926F927F928F929F92AF92BF9225
:10140000CF92DF92EF92FF920F931F93CF93DF93D0
:10141000CDB7DEB729970FB6F894DEBF0FBECDBFAC
:10142000A82E2B013A01490160E070E08EEB0E948A
:101430009406EE24FF2408E0B02E6E010894C11C2F
:10144000D11C87010C0D1D1D0E944406F8018083EC
:10145000BA940894E11CF11CB7FEEFCF69E070E08C
:10146000C6010E94D60B882319F083E090E009C0E2
:1014700084019301A201B6018A2D0E94B40780E085
:1014800090E029960FB6F894DEBF0FBECDBFDF9176
:10149000CF911F910F91FF90EF90DF90CF90BF9071
:1014A000AF909F908F907F906F905F904F90089536
:1014B000FF920F931F93CF93DF93EC01162F042F0E
:1014C000F22E0E9461050E94BD05882399F0BE019D
:1014D0008EE40E949406812F0E943206802F0E9483
:1014E00032068881883219F48F2D0E94320680E0FE
:1014F00090E006C082EB94E00E94940B81E090E0C3
:10150000DF91CF911F910F91FF9008950F931F933B
:10151000CF93DF93EC018B010E9461050E94BD0512
:10152000882379F0BE018EEB0E949406E80118E052
:101530000E9444068993115017FFFACF80E090E093
:1015400006C08DED94E00E94940B81E090E0DF9165
:10155000CF911F910F9108951F93CF93DF93182F71
:10156000EB010E9461050E94BD058823A9F0BE0120
:1015700088E40E949406113011F00E94C70562E1D0
:1015800074E380E090E00E94B306113011F00E94F5
:10159000DA0580E090E006C087E095E00E94940BB9
:1015A00082E090E0DF91CF911F910895CF93DF9378
:1015B000EC010E9461050E94BD05882369F0BE010F
:1015C00088EB0E94940662E174E380E090E00E9460
:1015D000B30680E090E006C081E395E00E94940BA2
:1015E00081E090E0DF91CF9108951F920F920FB6A6
:1015F0000F9211242F938F939F93EF93FF939BB19F
:101600002CB19871E091AC00EF5FEF718091AD006B
:10161000E81711F492E006C0E093AC00FF27E6570C
:10162000FF4F20839093AE00FF91EF919F918F9198
:101630002F910F900FBE0F901F9018951F920F9231
:101640000FB60F9211248F939F93EF93FF93909176
:10165000AA008091AB00981769F08091AB008F5F72
:101660008F718093AB00E82FFF27E659FF4F8081F1
:101670008CB901C05598FF91EF919F918F910F9078
:101680000FBE0F901F9018959C011092AA00109207
:10169000AB001092AC001092AD00832F992780BD53
:1016A00029B988E98AB986E880BD08959091AC008F
:1016B0008091AD00981719F480E091E00895809131
:1016C000AD008F5F8F718093AD00E82FFF27E65745
:1016D000FF4F20818091AE009927982F8827820F95
:1016E000911D08950895282F9091AA009F5F9F71E2
:1016F0008091AB009817E1F3E92FFF27E659FF4FE0
:1017000020839093AA00559A0895CF93DF93EC011C
:101710008881882331F089910E94730B8881882306
:10172000D1F7DF91CF910895CF93DF93EC01FC01C6
:1017300021968491882339F00E94730BFE01219633
:1017400084918823C9F7DF91CF910895CF93DF93D8
:10175000CDB7DEB761970FB6F894DEBF0FBECDBF31
:101760004AE050E0BE016F5F7F4F0E94F60B0E947F
:10177000850B61960FB6F894DEBF0FBECDBFDF912B
:10178000CF9108958F708A3010F0895C01C0805D20
:101790000E94730B08951F93182F82958F700E94DB
:1017A000C20B812F0E94C20B1F91089530E040E0D0
:1017B00050E046175707B9F0B8E1FC012081A8E0D6
:1017C000832F8227982F917080FD3B27369591308B
:1017D00009F430682695A15099F74F5F5F4F319615
:1017E0004617570759F7832F99270895E62FF72FA4
:1017F0002E2F3F2FE8944230CCF04532BCF44A30D3
:1018000029F497FB1EF4909581959F4F642F7727BD
:101810000E942B0C805D8A330CF0895D8193862FAA
:10182000972F009799F716F45DE25193932F822F2B
:1018300010820C941B0CDC01FC0101900020E9F7E4
:101840003297AE17BF0730F47C9160817083319777
:101850006D93F7CF0895AA1BBB1B51E107C0AA1FC8
:10186000BB1FA617B70710F0A61BB70B881F991F41
:101870005A95A9F780959095BC01CD01089597FBE5
:10188000092E07260AD077FD04D0E5DF06D0002018
:101890001AF4709561957F4F0895F6F790958195AC
:0418A0009F4F0895B9
:0A18A4000D0001030406090B0C0EF1
:00000001FF
